:100000008316003085008600831231288514851000
:1000100000308600190898002120980B0C287F30AA
:1000200086002520080080309C008514851005304E
:1000300099002E2005100514990B19289C0B1528E2
:100040000800051000000514080003309A009B0BFF
:1000500027289C0B27289A0B272808009B0B2E2863
:10006000080005309900851485107F308600252012
:10007000003086002120990B352803309900062096
:10008000990B3F2885148510252001308600031028
:100090001320860D861F4828203086001320860CEA
:0800A000061C4E281320312834
:00000001FF
